gpasm-2.1.3 (Mar 12 2018)    mc30p6060_lvd.asm  2018-5-14  11:00:04          PAGE  1


LOC  OBJECT CODE     LINE SOURCE TEXT
  VALUE

                      00001 #include mc30p6060.inc
                      00001                 LIST
                      00002 ;mc30p6080.inc    Standard Header File, Version 1.00 by Sinomcu
                      00326                 LIST
                      00002 
                      00003         org     0x00
0000   2800           00004         goto    start
                      00005         
                      00006         org     0x08
0008                  00007 inte:   
0008   0000           00008         NOP 
0009   2800           00009         goto    inte
                      00010        
000A                  00011 start:
                      00012       ; fill  0x00,0x40
000A   0BFF           00013         movai   0xff
000B   1586           00014         movra   P1  
000C   1585           00015         movra   P0         
000D   0B1F           00016         movai   0x1F;设置P10-P14口为输入
000E   15C6           00017         movra   DDR1 
000F   0B00           00018         movai   0x00;设置P0输出
0010   15C5           00019         movra   DDR0         
0011   0B00           00020         movai   0x00
0012   158D           00021         movra   PUCON
                      00022         
0013   0B01           00023         movai   0x01
0014   1588           00024         movra   MCR 
                      00025         
0015   3006           00026         jbset   P1,0
0016   3C88           00027         bclr    MCR,1
0017   3406           00028         jbclr   P1,0
0018   3888           00029         bset    MCR,1
                      00030        
0019   3086           00031         jbset   P1,1
001A   3D08           00032         bclr    MCR,2
001B   3486           00033         jbclr   P1,1
001C   3908           00034         bset    MCR,2
                      00035         
001D   3106           00036         jbset   P1,2
001E   3D88           00037         bclr    MCR,3
001F   3506           00038         jbclr   P1,2
0020   3988           00039         bset    MCR,3 
                      00040                 
0021   3206           00041         jbset   P1,4
0022   3E08           00042         bclr    MCR,4
0023   3606           00043         jbclr   P1,4
0024   3A08           00044         bset    MCR,4     
                      00045         
                      00046 
0025                  00047 main_loop:
0025   3288           00048         jbset  MCR,5
0026   1C85           00049         comr   P0
0027   2000           00050         call   delay
0028   1C86           00051         comr    P1
                      00052         ;NOP
                      00053         ;nop
                      00054         ;nop
                      00055         ;nop
                      00056         ;NOP
                      00057         ;bclr           P1,5 
0029   2800           00058         goto   main_loop
                      00059         
002A                  00060 delay: 
002A   0000           00061         NOP
002B   0000           00062         NOP
002C   0000           00063         NOP
002D   0000           00064         NOP
002E   000C           00065         return   
                      00066         
                      00067         end
gpasm-2.1.3 (Mar 12 2018)    mc30p6060_lvd.asm  2018-5-14  11:00:04          PAGE  2


SYMBOL TABLE
  LABEL                             VALUE

DDR0                              00000045
DDR1                              00000046
FSR                               00000004
INDF                              00000000
INTECON                           0000000E
INTFLAG                           0000000F
KBIM                              00000009
MCR                               00000008
ODCON                             0000000C
P0                                00000005
P1                                00000006
PCL                               00000002
PCLATH                            0000000A
PDCON                             0000000B
PUCON                             0000000D
PWMCR                             00000048
STATUS                            00000003
T0CNT                             00000001
T0CR                              00000041
T1CNT                             0000004D
T1CR                              0000004C
T1DAT0                            0000004F
T1DAT1                            00000049
T1DAT2                            0000004A
T1LOAD                            0000004E
TM0CR                             0000004B
_CONFIG0                          00008000
_CONFIG1                          00008001
__30P011                          00000001
delay                             0000002A
inte                              00000008
main_loop                         00000025
start                             0000000A
BUZE                              T1CR,5
C                                 STATUS,0
DBLCK                             PWMCR,4
DC                                STATUS,1
DDR00                             DDR0,0
DDR01                             DDR0,1
DDR02                             DDR0,2
DDR03                             DDR0,3
DDR10                             DDR1,0
DDR11                             DDR1,1
DDR12                             DDR1,2
DDR13                             DDR1,3
DDR14                             DDR1,4
DDR15                             DDR1,5
DDR16                             DDR1,6
DDR17                             DDR1,7
EIS                               MCR,6
FSR0                              FSR,0
FSR1                              FSR,1
FSR2                              FSR,2
FSR3                              FSR,3
FSR4                              FSR,4
FSR5                              FSR,5
GIE                               INTECON,7
INDF0                             INDF,0
INDF1                             INDF,1
INDF2                             INDF,2
INDF3                             INDF,3
INDF4                             INDF,4
INDF5                             INDF,5
INDF6                             INDF,6
INDF7                             INDF,7
INTIE                             INTECON,2
INTIF                             INTFLAG,2
INTOM                             T0CR,6
KBIE                              INTECON,1
KBIF                              INTFLAG,1
KBIM0                             KBIM,0
KBIM1                             KBIM,1
KBIM2                             KBIM,2
KBIM3                             KBIM,3
KBIM4                             KBIM,4
KBIM5                             KBIM,5
KBIM6                             KBIM,6
KBIM7                             KBIM,7
LVDEN                             MCR,0
LVDF                              MCR,5
LVDSEL0                           MCR,1
LVDSEL1                           MCR,2
LVDSEL2                           MCR,3
LVDSEL3                           MCR,4
P00D                              P0,0
P00PD                             PDCON,0
P01D                              P0,1
P01PD                             PDCON,1
P02D                              P0,2
P02PD                             PDCON,2
P03D                              P0,3
P03PD                             PDCON,3
P10D                              P1,0
P10OD                             ODCON,0
P10PD                             PDCON,4
P10PU                             PUCON,0
P11D                              P1,1
P11OD                             ODCON,1
P11PD                             PDCON,5
P11PU                             PUCON,1
P12D                              P1,2
P12OD                             ODCON,2
P12PD                             PDCON,6
P12PU                             PUCON,2
P13D                              P1,3
P13PU                             PUCON,3
P14D                              P1,4
P14OD                             ODCON,4
P14PU                             PUCON,4
P15D                              P1,5
P15OD                             ODCON,5
P15PU                             PUCON,5
P16D                              P1,6
P16OD                             ODCON,6
P16PU                             PUCON,6
P17D                              P1,7
P17OD                             ODCON,7
P17PU                             PUCON,7
PC0                               PCL,0
PC1                               PCL,1
PC2                               PCL,2
PC3                               PCL,3
PC4                               PCL,4
PC5                               PCL,5
PC6                               PCL,6
PC7                               PCL,7
PCH0                              PCLATH,0
PCH1                              PCLATH,1
PD                                STATUS,3
PMW0OE                            PWMCR,7
PMW1E                             PWMCR,1
PWM0E                             T1CR,6
PWM1OE                            PWMCR,6
PWM2E                             PWMCR,0
PWM2OE                            PWMCR,5
PWMINV                            PWMCR,2
PWMMD                             PWMCR,3
RST                               STATUS,7
T0C0                              T0CNT,0
T0C1                              T0CNT,1
T0C2                              T0CNT,2
T0C3                              T0CNT,3
T0C4                              T0CNT,4
T0C5                              T0CNT,5
T0C6                              T0CNT,6
T0C7                              T0CNT,7
T0IE                              INTECON,0
T0IF                              INTFLAG,0
T0PR0                             T0CR,0
T0PR1                             T0CR,1
T0PR2                             T0CR,2
T0PTA                             T0CR,3
T0PTS                             T0CR,5
T0SE                              T0CR,4
T1C0                              T1CNT,0
T1C1                              T1CNT,1
T1C2                              T1CNT,2
T1C3                              T1CNT,3
T1C4                              T1CNT,4
T1C5                              T1CNT,5
T1C6                              T1CNT,6
T1C7                              T1CNT,7
T1DAT00                           T1DAT0,0
T1DAT01                           T1DAT0,1
T1DAT02                           T1DAT0,2
T1DAT03                           T1DAT0,3
T1DAT04                           T1DAT0,4
T1DAT05                           T1DAT0,5
T1DAT06                           T1DAT0,6
T1DAT07                           T1DAT0,7
T1DAT10                           T1DAT1,0
T1DAT11                           T1DAT1,1
T1DAT12                           T1DAT1,2
T1DAT13                           T1DAT1,3
T1DAT14                           T1DAT1,4
T1DAT15                           T1DAT1,5
T1DAT16                           T1DAT1,6
T1DAT17                           T1DAT1,7
T1DAT20                           T1DAT2,0
T1DAT21                           T1DAT2,1
T1DAT22                           T1DAT2,2
T1DAT23                           T1DAT2,3
T1DAT24                           T1DAT2,4
T1DAT25                           T1DAT2,5
T1DAT26                           T1DAT2,6
T1DAT27                           T1DAT2,7
T1IE                              TM0CR,1
T1IF                              TM0CR,0
T1LOAD0                           T1LOAD,0
T1LOAD1                           T1LOAD,1
T1LOAD2                           T1LOAD,2
T1LOAD3                           T1LOAD,3
T1LOAD4                           T1LOAD,4
T1LOAD5                           T1LOAD,5
T1LOAD6                           T1LOAD,6
T1LOAD7                           T1LOAD,7
T1PR0                             T1CR,0
T1PR1                             T1CR,1
T1PR2                             T1CR,2
T1PTS0                            T1CR,3
T1PTS1                            T1CR,4
TBS                               TM0CR,7
TC1EN                             T1CR,7
TO                                STATUS,4
WDTEN                             MCR,7
Z                                 STATUS,2

Errors   :     0
Warnings :     0 reported,     0 suppressed
Messages :     0 reported,     0 suppressed

